:1000000000C90000000D000010D200000000000038
:1000100000000000000000000000000000000000E0
:100020000230059001E07401F02200022AA80102CA
:10003000200101022DDB0238B0000002081ED2AF01
:10004000320000021F19D2AF320000020826E490ED
:1000500001B9F0A3F012247690018112100312343A
:1000600077E4FCFD120E8590018112100F9001853E
:10007000E475F001120DEDC3900188E094649001E5
:1000800087E094005003020AD4900181120FF7EC2C
:10009000C0E0EDC0E0EEC0E0EFC0E0900185E0FE22
:1000A000A3E0FBEEFAE4F9F8D0E0FFD0E0FED0E008
:1000B000FDD0E0FC120F2B90018112100F900181F6
:1000C000120FF790017FEEF0A3EFF0A312101B00C8
:1000D0000000009001851234AC9001E1E07002A3B1
:1000E000E06003020AD4900189E07002A3E060039B
:1000F000020AD490013CE0700302096E90017BE09B
:100100007002A3E0701D90017FE0FFA3E090017BEF
:1001100012345B1234B590018B7403F0A374E8F0D1
:1001200002097E90017FE0FEA3E0FFC390017CE026
:100130009FFF90017BE09EFE1239289001A11210D2
:1001400058EE8FF0120E66900179E0701D9001A1BB
:10015000123463C39406E5F0940050081234601220
:1001600034B580069001797401F090017FE0FEA320
:10017000E0FFD390017CE09F90017BE09E4007E48C
:1001800090017AF0801890017A7401F0801090014B
:100190007B1234AC900179F090018D1234AD900156
:1001A00079E07003020AD4D390017EE094009001BC
:1001B0007DE094005003020AD4123460FF90017D68
:1001C000E0FCA3E0FDC3EF9DFFE5F09CFE123928A3
:1001D0009001BBEEF0A3EFF0A3E4F074C812345E1C
:1001E000D39494E5F09411400A9001BD7403F0A3F8
:1001F0007420F09001BBE0FFA3E09001A512345BF6
:10020000D312346A400CD39001BCE094641234964B
:10021000501312346012346950369001BCE094C817
:10022000123496402BE4900179F090017BF0123467
:100230005E1234699001895008E4F0A374C8F0801C
:10024000077401F0A3742CF0E490017AF0020AD450
:10025000123460FFD312346B404AD31234904044BE
:1002600090010812105874FF75F0F9120E2E9001CB
:100270008FE475F007120DEDC390018EE094E890C5
:10028000018DE09403501DA3E0940790018DE0944C
:1002900000400A74FF75F0F9120DED8007E490013B
:1002A0008DF0A3F01234601234695048123490403B
:1002B00043900108121058E475F007120E2E9001B9
:1002C0008DE475F007120DEDC3900190E094589005
:1002D000018FE09402501DA3E0940790018FE094F9
:1002E00000400A74FF75F0F9120DED8007E49001EB
:1002F0008FF0A3F090013CE0601B9001AFE0700232
:10030000A3E0701190011DE0FFA3E09001AFCFF0DA
:10031000A3EFF0801F90013CE07019123460C39489
:1003200096E5F09400500DE49001AFF0A3F0900139
:10033000B3F0A3F09001AFE07002A3E07003020BF2
:10034000DC123477C39001B0E09FFF9001AFE09ED4
:10035000FE1239289001B9EEF0A3EFF0123477D3F2
:100360009001B0E09F9001AFE09E400D9001B9E098
:10037000FFA3E09001B1CF801A9001B9E0FEA3E0A5
:10038000FFD394C8EE9400400EEE13FEEF13FF90DF
:1003900001B1EEF0A3EFF0D39001B2E0940A900126
:1003A000B1E094004056123460D39488E5F0941381
:1003B00040239001B4E094DC9001B3E09405503CFC
:1003C0009001B2E025E0FE9001B1E0339001B3F07E
:1003D000A3CEF08027123460D394E8E5F094034074
:1003E0001B9001B4E094F49001B3E09401500D909F
:1003F00001B1E0FFA3E0A3CFF0A3EFF09001F4E0A0
:1004000064016003020CAE90013CE06003020C9EAC
:10041000123477C3900196E09F900195E09E5004BE
:10042000EE12348890019BE07002A3E070671234F2
:1004300077D3900198E09F900197E09E4012900141
:1004400098E09FFF900197E09E900199F0A3EFF054
:10045000D390019AE09404900199E094004008122E
:10046000349D7464F08015D390019AE09406900155
:1004700099E09400400612349D74C8F090019B747A
:1004800003F0A374E8F090011DE0FFA3E090019752
:10049000CFF0A3EFF090019DE07002A3E0700F1287
:1004A0003480E490019FF0A3F09001B5801D90018D
:1004B0009FE0FFA3E09001B5CFF0A3EFF02212344C
:1004C00080E49001B5F0A3F090019FF0A3F022E743
:1004D00009F608DFFA8046E709F208DFFA803E886D
:1004E000828C83E709F0A3DFFA8032E309F608DFA4
:1004F000FA8078E309F208DFFA807088828C83E35F
:1005000009F0A3DFFA806489828A83E0A3F608DF1A
:10051000FA805889828A83E0A3F208DFFA804C804F
:10052000D280FA80C680D4806980F28033801080C7
:10053000A680EA809A80A880DA80E280CA80338927
:10054000828A83ECFAE493A3C8C582C8CCC583CC65
:10055000F0A3C8C582C8CCC583CCDFE9DEE7800D37
:1005600089828A83E493A3F608DFF9ECFAA9F0ED17
:10057000FB2289828A83ECFAE0A3C8C582C8CCC575
:1005800083CCF0A3C8C582C8CCC583CCDFEADEE843
:1005900080DB89828A83E493A3F208DFF980CC8828
:1005A000F0EF60010E4E60C388F0ED2402B4040049
:1005B00050B9F582EB2402B4040050AF23234582E6
:1005C00023900CFF73EF8DF0A4A8F0CF8CF0A4283B
:1005D000CE8DF0A42EFE22C2D5EC30E709B2D5E4D0
:1005E000C39DFDE49CFCEE30E715B2D5E4C39FFF4C
:1005F000E49EFE1210C3C3E49DFDE49CFC80031244
:1006000010C330D507C3E49FFFE49EFE22C5F0F877
:10061000A3E028F0C5F0F8E582158270021583E0AA
:1006200038F022BB010A89828A83E0F5F0A3E02238
:10063000500687F009E71922BBFE07E3F5F009E34E
:10064000192289828A83E493F5F074019322BB0115
:100650000789828A83020DED500B09C5F027F7C583
:10066000F01937F722BBFE0D09F8E325F0F3C5F0CA
:1006700019E338F322F889828A8374019325F0C53F
:10068000F0F8E4933822BB010A89828A83F0E5F00E
:10069000A3F0225006F709A7F01922BBFE06F3E5E6
:1006A000F009F31922EF2BFFEE3AFEED39FDEC389D
:1006B000FC22C3EF9BFFEE9AFEED99FDEC98FC2225
:1006C000E88FF0A4CC8BF0A42CFCE98EF0A42CFCD9
:1006D0008AF0EDA42CFCEA8EF0A4CDA8F08BF0A457
:1006E0002DCC3825F0FDE98FF0A42CCD35F0FCEBB6
:1006F0008EF0A4FEA9F0EB8FF0A4CFC5F02ECD397B
:10070000FEE43CFCEAA42DCE35F0FDE43CFC227571
:10071000F008758200EF2FFFEE33FECD33CDCC33E2
:10072000CCC58233C5829BED9AEC99E58298400C4A
:10073000F582EE9BFEED9AFDEC99FC0FD5F0D6E428
:10074000CEFBE4CDFAE4CCF9A88222B800C1B9000E
:1007500059BA002DEC8BF084CFCECDFCE5F0CBF96F
:100760007818EF2FFFEE33FEED33FDEC33FCEB3367
:10077000FB10D703994004EB99FB0FD8E5E4F9FA95
:10078000227818EF2FFFEE33FEED33FDEC33FCC97A
:1007900033C910D7059BE99A4007EC9BFCE99AF90D
:1007A0000FD8E0E4C9FAE4CCFB2275F010EF2FFF7C
:1007B000EE33FEED33FDCC33CCC833C810D7079BE6
:1007C000EC9AE899400AED9BFDEC9AFCE899F80F49
:1007D000D5F0DAE4CDFBE4CCFAE4C8F922EB9FF5DE
:1007E000F0EA9E42F0E99D42F0EC6480C864809893
:1007F00045F022EB9FF5F0EA9E42F0E99D42F0E8D9
:100800009C45F022E8600FECC313FCED13FDEE13E2
:10081000FEEF13FFD8F122E0FCA3E0FDA3E0FEA36E
:10082000E0FF22E0F8A3E0F9A3E0FAA3E0FB22EC6A
:10083000F0A3EDF0A3EEF0A3EFF022A8828583F001
:10084000D083D082121032121032121032121032B3
:10085000E473E493A3C583C5F0C583C8C582C8F01B
:10086000A3C583C5F0C583C8C582C822A42582F567
:1008700082E5F03583F58322E0FBA3E0FAA3E0F9FB
:1008800022EBF0A3EAF0A3E9F022EC8EF0A4CCC5B1
:10089000F0CCCDF8EFA4CEC5F02DFDE43CFCE8A4EF
:1008A0002EC8C5F03DFDE43CFCEFA4FFE5F028FEBA
:1008B000E43DFDE43CFC22EF4E6012EF60010EEDE2
:1008C000BB010B89828A83F0A3DFFCDEFA2289F068
:1008D0005007F709DFFCA9F022BBFEFCF309DFFC9F
:1008E000A9F022BC000BBE0029EF8DF084FFADF013
:1008F00022E4CCF875F008EF2FFFEE33FEEC33FC6A
:10090000EE9DEC984005FCEE9DFE0FD5F0E9E4CE9F
:10091000FD22EDF8F5F0EE8420D21CFEADF075F06E
:1009200008EF2FFFED33FD4007985006D5F0F22277
:10093000C398FD0FD5F0EA22208A03021508900122
:1009400079E060030215089001E3E07002A3E06023
:10095000030215089001E1E07002A3E060030215B4
:1009600008900166E07002A3E06003021508122FF0
:1009700062600302150890013CE0FF600302150865
:10098000EF7038900117122F02900105122EFFD33D
:100990009FE5F09E40030215087E007F0A7D007BE4
:1009A000017A01793D121097E4900172F0A3F09062
:1009B00001E9F0A3F09001E7F0A3F0E4F5B29001B3
:1009C00076E0FFA3E090021ACFF0A3EFF0C20B3065
:1009D00004030214DD758D20438D20758D8043A89E
:1009E00008D2AF758B02758EC820042B122F62704F
:1009F00026200923E5DB5404701D758AA420091301
:100A0000E5DB5404700DF5867587030000007586DC
:100A1000018006D20B8002D20B758B01758A305390
:100A2000A8F7D39001E2E094909001E1E0940140B6
:100A30000A74FE75F070120DED8007E49001E1F08C
:100A4000A3F0D39001EEE094909001EDE09401408A
:100A50000A74FE75F070120DED8007E49001EDF060
:100A6000A3F0E490021EF0A3F0121AD290015EEE01
:100A7000F0A3EFF0900162EEF0A3EFF0C390021B41
:100A8000E09FFF90021AE09EFE12392890021CEEB1
:100A9000F0A3EFF0D39414EE94005025A3E475F086
:100AA00001120DEDD390021FE0940590021EE09418
:100AB000004002D20BD390021DE0940F122F285059
:100AC000A8122F2140030214CD300B030214CD9045
:100AD0000156E0FEA3E0FF900162E0FCA3E0FD9F71
:100AE000EC9E402BED9FFFEC122F127FB87E8812F8
:100AF0002F2F400912101B0000EA60804F120FF7E1
:100B0000EF24A8FFEE3461FEE43DFDE43C80399023
:100B10000162E0FEA3E0FFC3900157E09FFF900158
:100B200056E0122F127FA87E61122F2F400912105B
:100B30001B000000008015121003C374A89BFF74F3
:100B4000619AFEE499FDE498FC122F1B9001BB1200
:100B50000FF79001B9EEF0A3EFF090021AE0FEA3B8
:100B6000E0FF7C007D0912106AECF8EDF9EEFAEF77
:100B7000FB900162E0FEA3E0FFE4FCFD120E857B2A
:100B80000A122EF890021AEEF0A3EFF090013CE06A
:100B9000704A900108122F02FFAEF0122ED9900178
:100BA00000EEF0A3EFF0900108122F02FFAEF07CF0
:100BB000007D0312106A900100122EE390010812CA
:100BC0002F09900100E0FEA3E0FF122F089001051D
:100BD000122F6990010E122F690214CD900100E0CE
:100BE000FEA3E0FF122ED9900100EEF0A3EFF01269
:100BF0002F08900108122F02FFD39001BAE09F90B6
:100C000001B9E095F050030214DD120E03900102C9
:100C1000122EFF122F5AC3EF9515EE9514500302B2
:100C200014DD900105122F02FFAEF07C007D021250
:100C3000106AECC0E0EDC0E0EEC0E0EFC0E0900173
:100C400008122F02FFAEF0900102122F02122F5A4B
:100C5000E4FCFDD0E0FBD0E0FAD0E0F9D0E0F812FF
:100C60000E85E47B03122EF9900105122F099001E5
:100C700005122F02D39430E5F09475400874757511
:100C8000F030120E66900179E0606290017DE0FE26
:100C9000A3E0FFD39400EE94004052900105122F80
:100CA00002122F5A1239289001BFEEF0A3EFF090F4
:100CB0000105122F02C3122F405012122F4D400D6A
:100CC000900108121058E475F007120E2E900105DD
:100CD000122F02D3122F404014D3122F4D400E90EA
:100CE000010812105874FF75F0F9120E2E200B0D2A
:100CF000122F215008122F6270030211AF90017859
:100D0000E004F090018112101B00000000E490014B
:100D100085F0A3F0A3F0A3F09001FB12101B0000DC
:100D200000001238B01237FA22122C6E400302175C
:100D3000FA900108122C37FDE5F0FC122C34FFAEBE
:100D4000F0D39DEE9C402E122CCDD3EF9430EE9438
:100D500075400C9001B97475F0A37430F0801012D6
:100D60000E03C39DFEE5F09C9001B9F0A3CEF0E424
:100D70009001A78060120E03FFAEF0C3ED9FFBEC65
:100D80009EFAD3EB9410EA9427400C9001B9742793
:100D9000F0A37410F08009C3ED9FFFEC9E122C8A23
:100DA0009001B9E0FFA3E09001A7CFF0A3EFF030EE
:100DB0000018D3E0942C9001A7E094014013900117
:100DC000A97427F0A37410F08007E49001A9F0A3A0
:100DD000F0E49001B9F0A3F090013CE0604A122CDD
:100DE0003DD39400EE648094804014D3EF9509EED7
:100DF0009508400B9001E7E4F0A37464F0801BD3E6
:100E00009001E8E094009001E7E09400400C90012C
:100E100005122C37FFE5F0122C8AD2089001ED74F0
:100E20000FF0A374A0F0800F9001EB7403F0A37493
:100E3000E8F0E4FF123756D39001BAE09400900135
:100E4000B9E06480948050030217CFE0FEA3E0FF76
:100E5000900105122C2B122C3DEE3395E0FDFCE4A5
:100E60007BB87A88F9F8C3120FBD500A9001B974A3
:100E700088F0A374B8F0D39001EAE094009001E9FF
:100E8000E0940050089000F1E06420702AE5092405
:100E90000AFFE43508FE9001B9E0FCA3E0FDC39F22
:100EA000EC9E5013ED9400EC648094804038122C3A
:100EB0003D7C007D0A802930002C90013CE07011BF
:100EC000122C3DC39515EE9514501B7C027DBC8001
:100ED0000F122C3DC39509EE9508500A7C027DBC8B
:100EE000120DB7122C8990013CE070030217549048
:100EF00001EBE07002A3E070149001B9E0FEA3E002
:100F0000FDEEFCE4FF1217FB122C898035122C3DFC
:100F1000C3900135E09FFF900134E09EFE12392816
:100F2000D3EF9428EE648094804017D39001ECE0D6
:100F300094C89001EBE09400400874FF75F09C1297
:100F40000DED900134E0FEA3E0FF7C007D0F121058
:100F50006AECF8EDF9EEFAEFFB122C3DEE3395E07A
:100F6000FDFC120E85E47B10FAF9F8120F2B9001AC
:100F700034EE800B9001B9E0FFA3E0900134CFF094
:100F8000A3EFF0900134E0FEA3E0FFD39405EE94CC
:100F900000400EEF9410EE940050069001B9EE80E0
:100FA00016900130E0FEA3E0FF900135E02FFF90A6
:100FB0000134E03E9001B9F0A3EFF0D39001BAE024
:100FC00094309001B9E0648094F540077475F0A303
:100FD0007430F0E5DB54047041122C3D90010E1288
:100FE0002C2B9001BAE024A8FF9001B9E08022E503
:100FF000DB54047025122C58900130E0FEA3E0FF72
:1010000090010E122C2B90010E122C3724A8FFE514
:10101000F03461FE90010B122C2B229001BBEFF0FB
:10102000A3ECF0A3EDF0EF122BE0E0FEA3E0C39DF4
:10103000FFEE9CFE123928D3EF9428EE6480948052
:10104000401C122BB012101B00000000122B7CE47D
:10105000F0122BFA122BDCEEF0A3EFF0803B122BF8
:101060006B122C1040339001BCE0FCA3E0FDD3EFE9
:101070009DEE9C400B9001BBE0122BA3E04401F0DD
:101080009001BBE0FF122B6FE0FAA3E0C39DEA9C46
:101090005007122BA2E04402F09001BBE0122BB5E6
:1010A000C083C082121003122BFAE4FCFD120E85DD
:1010B000D082D08312100F9001BBE0FF122C03E40A
:1010C00075F001120DEDEF75F007A42443F582E4ED
:1010D0003439F583E493FE740193FF9001BBE0FD86
:1010E000C454F02412F582E43402F583E0FAA3E05C
:1010F000C39FEA9E5003021A67ED122C03E0FEA381
:10110000E0FFFBEEFAE4F9F89001BBE0122BB51218
:101110000FF7120F2B9001BE12100F122B65E0FC7F
:10112000A3E0C39FFFEC9EFE1239289001C2EEF0AF
:10113000A3EFF09001BBE0FD75F007A4243EF5821B
:10114000E43439F583C37401939FE4939E401FED0B
:10115000122B6FE0FEA3E04E60149001BBE0FB1287
:101160002BEDE0FEA3E0C394B8EE940B501E90016B
:10117000BBE0FF122B6FE0FCA3E04C7008EF122BDA
:10118000EDE4F0A3F0122B65EE021A0EEB60030201
:101190001A149001C4F09001C2E0FEA3E0FFD394C2
:1011A00050EE94004006A37408F080329001BBE03A
:1011B000122BA3E064036026D3EF943CEE9400402E
:1011C000089001C47404F08015D39001C3E0942802
:1011D0009001C2E0940040069001C47402F0122B0A
:1011E0006BE0FEA3E0FFE4FCFD122C1CD3120FD336
:1011F00040119001C4E0FF122B6BE48FF0120DED53
:10120000021A4AD39001C3E094509001C2E09400C6
:101210004058122B6BC083C082E0FEA3E0FF900118
:10122000C4E0FDC3EF9DFFEE9400D082D083F0A315
:10123000EFF08036122B6BE0FEA3E0FF4E700D1234
:101240002C1CEBFFEAFEE9FDE8FC80167C007D0724
:1012500012106A122C1C120E85E47B08FAF9F8129F
:101260000F2B122B6BEEF0A3EFF0122BB012101B12
:1012700000000000122B7CE4F09001BE120FF71268
:101280002BDCEEF0A3EFF0122B6B122C10405F90D2
:1012900001BDE09FFF9001BCE09EFE123928900145
:1012A000BBE075F007A42440F582E43439F583D31C
:1012B0007401939FE4939E400F9001BBE0FF122BBB
:1012C0006F122BC2E4F080269001BBE0FF75F0079F
:1012D000A42442F582E43439F583E493FE122BCE44
:1012E000E0C39E5009122B6B122BC2E004F0122BAC
:1012F000FA229001C712101B00002710E4FF1233DE
:1013000017E49001C4F09001C4E0FF7E00C394068E
:10131000748094804003021C0DEF2401FFEE33FE25
:1013200012358DFDD3EF9D7480F86E984003021C3A
:1013300004E4FF123893758A50902E207401F090C7
:101340002E20E030E2F99001F4E09008119375F05E
:1013500002902E0012104CE0FFA3E09001C5CFF0E8
:10136000A3EFF0902E20E4F0758A30FF12390B9035
:101370000191E0FEA3E0FF9001C6E02FFF9001C5C0
:10138000E03EFE900193E0FCA3E0FDC3EF9DFFEE85
:101390009CFE9001C5F0A3EFF09001ADEEF0A3EF3D
:1013A000F0900158E0FEA3E0FF4E700E9001ADE01A
:1013B000FCA3E0FDECFEEDFF801E7C007D03120D22
:1013C000A59001AEE02FFF9001ADE03EFE7802EF68
:1013D000CEC313CE13D8F9FF900158EEF0FAA3EF65
:1013E000F0FB12359FFFE4FCFD9001CC12100FEBD7
:1013F000FFEAFEE4FCFD9001D012100FE4FF122082
:101400008C90015CEEF0A3EFF09001F4E0640190A9
:1014100001C712359C2400FFEE34E8FE3395E0FD51
:10142000FC1235BB9001C4E004F0021AE6902E23B2
:10143000E4F09001C7121003E8C0E0E9C0E0EAC0A0
:10144000E0EBC0E012358DFFFBE4FAF9F81235B598
:10145000123655D0E0FBD0E0FAD0E0F9D0E0F81237
:1014600035BBE47F507EC3FDFC9001C7121003D34F
:10147000120FBD400A9001C712101B0000C350128A
:1014800035B5EC33500A9001C712101B0000000064
:10149000900160E0FAA3E0FB4A70051235B58022A6
:1014A0007E007F02EBFDEAFC12106AECF8EDF9EE2B
:1014B000FAEFFB1235B5120E85E47B03FAF9F81248
:1014C0000F2B900160EEF0A3EFF0900156E0700258
:1014D000A3E0700F900160E0FFA3E0900156CFF011
:1014E000A3EFF090012612359CFFE4FCFD120E855F
:1014F00090012612100F90012AE475F001120DEDF3
:1015000090012AE0FEA3E0FFD3940AEE9400402964
:10151000EFFBEEFAE4F9F8900126120FF7120F2B09
:10152000900124EEF0A3EFF0E490012AF0A3F090F4
:10153000012612101B0000000090012CE07002A395
:10154000E0703A900124E0FEA3E0FFC390015DE06B
:101550009FFF90015CE09EFE123928900122EEF080
:10156000A3EFF0D39406EE9400401290012C740384
:10157000F0A374E8F0A3E475F001120DED900160A2
:10158000E0FEA3E0FF22D39001E2E09F9001E1E0C2
:101590009E400AA3E09FF09001E1E09EF09001E6FA
:1015A000122D8B9001E5E09C400CA3E09FF0900190
:1015B000E5E09EF08002D28AD39001E4E09F9001A2
:1015C000E3E09E400AA3E09FF09001E3E09EF0126A
:1015D0002D9D5003122DD5D39001E8E09F9001E797
:1015E000E09E400AA3E09FF09001E7E09EF0D390D8
:1015F00001EAE09F9001E9E09E400AA3E09FF0909D
:1016000001E9E09EF0D39001F0E09F9001EFE09EB1
:10161000400AA3E09FF09001EFE09EF0D39001EC30
:10162000E09F9001EBE09E400AA3E09FF09001EB69
:10163000E09EF0D39001EEE09F9001EDE09E400A25
:10164000A3E09FF09001EDE09EF0D39001AAE09F0F
:101650009001A9E09E400AA3E09FF09001A9E09EBE
:10166000F0D39001F2E09F9001F1E09E400AA3E0E8
:101670009FF09001F1E09EF0122DAB5003122DD59A
:10168000D390018AE09F900189E09E400AA3E09FE9
:10169000F0900189E09EF090018C122D8B90018BCF
:1016A000E09C400AA3E09FF090018BE09EF0D39075
:1016B000019CE09F90019BE09E400AA3E09FF09078
:1016C000019BE09EF0D390019EE09F90019DE09EE3
:1016D000400AA3E09FF090019DE09EF0EF2401FD01
:1016E000E43EFCD3900167E09D900166E09C400AD7
:1016F000A3E09FF0900166E09EF0D39001ACE09FE4
:101700009001ABE09E400AA3E09FF09001ABE09E09
:10171000F0122DB95003122DD5122DC75003122DE2
:10172000D5D390012DE09F90012CE09E400AA3E0CC
:101730009FF090012CE09EF022C0E0C0F0C083C07A
:1017400082C0D0E8C0E0D2AFD39001E2E094009034
:1017500001E1E094004003122D84D39001E6E0946F
:10176000019001E5E094004005122D848002D28AA8
:10177000D39001E4E094009001E3E0940040031270
:101780002D84122D9D5003122D96D39001E8E094E4
:10179000009001E7E094004003122D84D39001EA09
:1017A000E094009001E9E094004003122D84D3906E
:1017B00001F0E094009001EFE094004003122D84CA
:1017C000D39001ECE094009001EBE0940040031210
:1017D0002D84D39001EEE094009001EDE094004060
:1017E00003122D84D39001AAE094009001A9E09403
:1017F000004003122D84D39001F2E094009001F197
:10180000E094004003122D84122DAB5003122D964C
:10181000D390018AE09400900189E0940040031283
:101820002D84D390018CE0940190018BE0940040D2
:1018300003122D84D390019CE0940090019BE094CE
:10184000004003122D84D390019EE0940090019DEE
:10185000E094004003122D84D3900167E09401903E
:101860000166E094004003122D84D39001ACE09413
:10187000009001ABE094004003122D84122DB9506A
:1018800003122D96122DC75003122D96D390012DC1
:10189000E0940090012CE094004003122D84D0E0ED
:1018A000F8D0D0D082D083D0F0D0E0329001CBEF0E
:1018B000F0122A21E070279001CBE0122A58120F73
:1018C000F7E4FBFAF9F8C3120FD360129001CBE0F2
:1018D000122A76120FF7E4F8C3120FD37057122AA8
:1018E0008A9001CC1221C8EEF0A3EFF0ED122A216C
:1018F000E06029ED75F00AA4243AF582E43439F564
:1019000083C083C0829001F4E0D082D083122A2F5A
:10191000400A9001CBE0122A217405F01229D6E08A
:10192000D39400748094804006122A20E014F09032
:1019300001D00221C4122A53120FF79001D41210C1
:101940000F122A75120FF79001D812100F9001CBC9
:10195000E0122A67120FF7EFF9122A93E9F8120F33
:10196000E4EFFBEEFAEDF9ECF8122A93120E9290E6
:1019700001DC12100F9001D4120FF79001D0121059
:1019800003120E859001DC121003120E85122A84B8
:10199000122A53122A90122A75122A90122A991288
:1019A0001003120F2B122A849001D81221C8EEF0D6
:1019B000A3EFF0ED75F00AA42436F582E43439F58E
:1019C00083C083C0829001F4E0D082D083122A2F9A
:1019D000400F1229D67405F0122A8A9001D81210ED
:1019E0000F9001D8120FF722EFFBEEFA120FF7C398
:1019F000EF9BFFEE9AFE1239289001CBE0FD75F0C7
:101A000013A42400F582E43402F5832290017212BB
:101A10002CD49404EE94005022122C9DEF25E0FF6C
:101A2000EE33FE746A2FF58274013EF583ECF0A369
:101A3000EDF0900172122CB10222B79001C6740130
:101A4000F09001C6E0FFC3122C675021EF122C7CEE
:101A5000FCA3E0FDEF25E02468F582E43401F58382
:101A6000ECF0A3EDF09001C6E004F080D490013CCE
:101A7000E060028053122C34FF122C9DC3EF9DFFB7
:101A8000E5F09CFE123928C3EF9428EE6480948020
:101A90005036900108122C37FFC3900101E09FFFE0
:101AA000900100E095F0FE123928C3EF9414EE6423
:101AB00080948050059001088003900102122C3719
:101AC000FF900170E5F0800B900100E0FFA3E09033
:101AD0000170CFF0A3EFF09001C212101B000000C4
:101AE00000E49001C6F09001C6E0FFD3900173E0DE
:101AF0009F900172E0940040259001C21210039063
:101B000001C6E0122C7CFEA3E0FFE4FCFD120E8572
:101B10009001C212100F9001C6E004F080C890013D
:101B2000C2120FF7ECC0E0EDC0E0EEC0E0EFC0E0A5
:101B3000900172122CB8D0E0FFD0E0FED0E0FDD0D2
:101B4000E0FC120F2B9001C212100F9001C2020F85
:101B5000F79001B97402F0A374BCF0D39001ACE02B
:101B600094009001ABE094004011122C34FF9001DE
:101B700008121058E5F08FF0120E669001E1E07047
:101B800002A3E0600B9001B9E4F0A37464F0800B51
:101B900090001AE0641170037420F090013CE06042
:101BA0000F7E007F0A7D007B017A01793D0210974C
:101BB00090013D121003E8C0E0E9C0E0EAC0E0EBAC
:101BC000C0E0122C34FFAEF0E4FCFDD0E0FBD0E02E
:101BD000FAD0E0F9D0E0F8120E8590013D12100F16
:101BE000900141122CB19001B9122CD4900146E021
:101BF0009F900145E09E500302247590013D120F15
:101C0000F7ECC0E0EDC0E0EEC0E0EFC0E0900141D5
:101C1000122CB8D0E0FFD0E0FED0E0FDD0E0FC1206
:101C20000F2B90013D12100F900108122C37243217
:101C3000FFE435F0FEE4FCFD90013D121003D312E9
:101C40000FD3402E9001E1E07002A3E07024200841
:101C500021900143122CB2D3900144E094059001ED
:101C600043E094004018122C22E4900143F0A3F0CA
:101C7000800C122C22E4900143F0A3F0C2089001E2
:101C80003D12101B00000000E4900141F0A3F09011
:101C90000145F0A3F022758D20438D20538D7FE404
:101CA000F5B275B6FF75B7FF75B2A243B20153A87E
:101CB000FB538B7F758B10438B08E58B20E703006C
:101CC00080F8538B7F758B11438B08E58B20E703DE
:101CD0000080F8900223E5B5F0A3E5B4F0758B0120
:101CE000E4F5B21238B0E4F58D90011DE0FEA3E0FA
:101CF000FF4E7010123849FD90011DE5F0F0A3ED84
:101D0000F0022566123849FDC3EF9DFFEE95F0FE07
:101D1000123928D3EF940AEE64809480402412385C
:101D200049FFC390011EE09F90011DE095F0500611
:101D3000E475F001800790011D74FFF5F0120DEDC0
:101D4000804490011DE0FEA3E0FF7C007D031210A3
:101D50006AECC0E0EDC0E0EEC0E0EFC0E012384950
:101D6000FFAEF0E4FCFDD0E0FBD0E0FAD0E0F9D02B
:101D7000E0F8120E85E47B04FAF9F8120F2B9001BB
:101D80001DEEF0A3EFF09001F4E06401700D7D2FE3
:101D90001238287002A3E0701A800B7D17123828C1
:101DA0007002A3E0700D900191E0FFA3E0A3CFF0DB
:101DB000A3EFF0900195E07002A3E0700F90011D79
:101DC000E0FFA3E0900195CFF0A3EFF0227FFF7A30
:101DD0000079001238E77FB97A0179001238E77E7E
:101DE000007F147D007B017A0179E0121097902D1D
:101DF000E0E493900001F09000047411F0A37422C9
:101E0000F0A37433F0902DE2E493900012F0902D43
:101E1000E3E493900014F09000FB7401F09000361E
:101E20007410F09000F1F0900024F0A37420F09072
:101E300000207410F07B017A0079409001021210AA
:101E4000617A0079449001081210617A0079429019
:101E500001051210617A00792E90010B1210617A3F
:101E600000792A90010E1210617A007928900111F0
:101E70001210617A00796090011F1210617A007966
:101E8000809001A11210617A007918900139121026
:101E9000617A00791B9001361210617A00793290D4
:101EA00001141210617A0079269001171210617ADC
:101EB00000793490011A121061900114121058E444
:101EC00075F0C8120E66900117121058E475F06490
:101ED000120E6690011A121058E475F096120E66F2
:101EE0007514007515C87508007509969001E174A0
:101EF00007F0A374D0F0E49001E0F0229001C0EF6D
:101F0000F0902E22E0FF9001C4E4F0A3EFF0758A78
:101F100050902E227401F012352D7404F0A3E4F0D9
:101F20009001C1F09001C1E0FFC3940D74809480D2
:101F300040030227F0EFF87E02E4088006CEA2E715
:101F400013CE13D8F8FF9001C2EEF0A3EFF04E705D
:101F5000079001C2F0A304F0902E207401F0902E9F
:101F600020E030E2F99001C0E0FF902E00123534FD
:101F7000E0FCA3E0D394FEEC94074040123555E01A
:101F8000FEA3E0FF9001C2E0FCA3E0FDEF2DFFEE19
:101F90003CFEC3EF94FFEE94079001C0E075F002A1
:101FA000902E10500B12104CEC8DF0120DED805055
:101FB00012104C7407F0A374FFF080449001C0E04D
:101FC000FF123531E0FCA3E0FD9001C2E0FAA3E08E
:101FD000FBD3ED9BEC9A4021123555C083C082C3E0
:101FE000A3E09BFF0582D5820215831582E09AD07B
:101FF00082D083F0A3EFF0800712352DE4F0A3F038
:10200000902E20E4F0F58D9001C1E004F002270449
:102010009001C4A3E0902E22F0758A30227FC87E02
:10202000007D967C00122C6E40030228EE300020CA
:102030009001A9E07002A3E060087514137515887B
:1020400080067514037515E8750803750920804925
:102050009001F4E0F964017006FE7FC8FC7D969063
:1020600001B3E0FAA3E0FB2FF515EA3EF514CEEC40
:10207000CEEDFFEB2FF509EA3EF508E96401701992
:10208000A3E0FEA3E0FF2515F515EE3514F514EFDA
:102090002509F509EE3508F508900105122C37FFE2
:1020A000AEF0C39515EE9514500F90013CE0601A08
:1020B000C3EF9509EE950840119001E9E07002A385
:1020C000E0702990013C04F080229000F1E064204F
:1020D0009001E97005F0A3F080077401F0A374F497
:1020E000F0E490013CF09001E7122CC390013CE039
:1020F000FF6016900024E0641090003670057410A4
:10210000F080037420F0122CA690004BEFF022E434
:10211000F526F525F524F523F526F525F524F523F3
:10212000F522122C64502AE52225E0240AF8E6FE66
:1021300008E6FFE4FCFDE5262FFFE5253EFEED3534
:1021400024FDEC35238F268E258D24F52305228052
:10215000D1E47B04FAF9F8AF26AE25AD24AC231206
:102160000F2B900176EEF0A3EFF0E47526A875250D
:1021700061F524F523F522122C6450559001761256
:102180002C46C3122CCD123928D3EF940AEE64806A
:1021900094804012900176E0FEA3E0FF900156E0AB
:1021A000FCA3E0FD8007900156122C46C3122CCDF3
:1021B0003395E0FDFCE5262FFFE5253EFEE5243DB9
:1021C000FDE5233C8F268E258D24F523052202294B
:1021D00057E47F607EEAFDFCAB26AA25A924A8234C
:1021E000D3120FD3400BE47526607525EAF524F56C
:1021F00023AE25AF26229001D0120FF79001CBE03D
:10220000FB75F013A424FBF582E43401F58312106E
:102210000FEB75F013A42406F582E43402F5831263
:102220000FF79001D0121003120EA09001CBE0FB2B
:1022300075F013A424F7F582E43401F58312100F2E
:10224000EB75F013A424FFF582E43401F5832275C5
:10225000F00212104CE493FE740193FFED75F0133D
:10226000A42400F582E43402F583E0FCA3E0D39FCC
:10227000EC9E229001CBE0FB75F013A424FBF582C9
:10228000E43401F58322EB75F013A42402F582E413
:102290003402F58322EB75F013A424F7F582E434BD
:1022A00001F583229001D812100F9001D0020FF790
:1022B00012100F9001D8020FF7EB75F013A424064B
:1022C000F582E43402F58322C0E0C083C082C0D02E
:1022D00075D018D2AFE5DB30E422D209C206E5DBC7
:1022E00030E11412391AE0F5DFEF64077065D28A25
:1022F000900007F0022B56C205022B59E5DB30E5B2
:102300002C9000F0E064AA7017758A10F5DAC2AF5D
:10231000F5B2F5A8F5A9F58B758E01758DC080FE17
:10232000D204300604C2068050C209804CC206E5C1
:10233000DB30E121E5DB30E04012391AE0F5DFEF78
:1023400024F9600824EE700BD20A8007D28A90002C
:1023500007E4F0802120050A7816A6DFD205D20610
:10236000801712391AE5DFF0EF642470099001E359
:1023700004F0A374F4F078160675DBFFD0D0D08299
:10238000D083D0E0329001BE120FF79001BBE0C4C1
:1023900054F02410F582E43402F58322EBC454F0A7
:1023A000240EF582E43402F583E4F0A3F09001BB3F
:1023B000E0FFC454F02412F582E43402F583E4F023
:1023C000A3F0EFC454F02417F582E43402F583221D
:1023D0009001BBE0FBC454F0240AF582E43402F51A
:1023E0008322E0FDA3E09001BCCDF0A3EDF0EFC4AB
:1023F00054F02416F582E43402F583229001BBE008
:10240000C454F02414F582E43402F58322C454F059
:102410002418F582E43402F583229001BCE0FEA387
:10242000E0FF22C454F0240EF582E43402F5832246
:10243000E0FEA3E0FFD39400EE9400229001BE02E0
:10244000100390013D120FF7900108121058EE8F03
:10245000F0020E66900102121058020E039001B9AC
:10246000E0FEA3E0FF22E52225E0240AF8E6FE08CC
:10247000E6FFE0FCA3E0FD22900105121058E4F510
:10248000F0020E66C3E52294047480948022D390F7
:1024900001E2E094009001E1E094002225E0246A4A
:1024A000F582E43401F583E022EE9001B9F0A3EF68
:1024B000F022121058746175F0A8020E66900100A7
:1024C000E0FCA3E0FD229001E37403F0A37420F08C
:1024D00022E475F001020DEDE0FEA3E0FBEEFAE46C
:1024E000F9F822F0A3F09000367410F022EF9DFF6F
:1024F000EE9CFE22E0FEA3E0FFC3221233871238D7
:10250000757E007F287D007B017A01797912109712
:1025100012082EE4900172F0A3F0900160F0A3F095
:1025200090015EF0A3F0900162F0A3F07F041231FD
:10253000A9900100E0FEA3E0FFA3122C2B90010064
:10254000E0FEA3E0FF122C28122C5890010B122C55
:1025500092900111122C9290010E122C5BE49001CA
:102560003CF0FE7F0AFD7B017A01793D121097E471
:102570009001EFF0A3F09001ED122CC3E490004B1A
:10258000F0122CA69001F3E0700FC39001E2E094EA
:10259000F49001E1E09401500A9001E17401F0A38C
:1025A00074F4F02274FFF5F0020DEDEF2401FDE468
:1025B0003EFCD3E09D22E475F001020DEDC39001D5
:1025C00046E094BC900145E0940222C3900188E06B
:1025D0009464900187E0940022C3900219E094B8BB
:1025E000900218E0940B22C3900213E094F490023E
:1025F00012E0940122EE8FF0020DEDD2AF32000016
:102600000D01ABC974AA7583F5758255A57455750E
:1026100083FA7582AAA574A57583F5758255A522DE
:102620000203030AB0B00BB6B60CFFFF09020208A2
:10263000FFFF0D77770E04041307071410101080A6
:1026400080150000160000019212071B1A0F0404E7
:10265000040101112018122418030202E49001B9A8
:10266000F0A3F0900149F0A3F09001477427F0A384
:102670007410F01236997E007F027D007B017A0192
:102680007956121097E4FF12371C12353A9001B9AF
:10269000CDF0A3EDF09001B9E0FCA3E0FDC39405FB
:1026A000EC94004009D3ED94F0EC94074017EF64EC
:1026B000014E70059001498004E4900147F0A3F0B9
:1026C000E4FF12371C902E23E4F012353A9001B942
:1026D000CDF0A3EDF090001D7410F0EF64014E906A
:1026E00001B9700812352112355F800612352112AA
:1026F0003569E03EFE123549227C007D0312106AE6
:102700009001B9ECF8EDF9EEFAEFFBE0FEA3E0FF83
:10271000E4FCFD120E857B04E4FAF9F8020F2BFFAE
:10272000AEF0121058020E03A3121058EE8FF002F2
:102730000E669EFE7C007D0412106A9001BB0210A2
:102740000FC390021DE0941490021CE0940022E458
:10275000FDFC9001BB121003D3120FD39001BB22DA
:10276000FF90017EE09F90017DE095F0229001C0F6
:10277000E0940A9001BFE0940022C39FFFE5F09E21
:10278000FE229000F1E0642022121058E4F5F002DD
:102790000E66900020E0642070037421F0900136F2
:1027A000121058120E03641045F070031235C490D5
:1027B0000001E064AA70031234C0900013E0FF7EB1
:1027C0000064107002D203EF64204E7002C2031244
:1027D00032A420070890001AE06410700B90001AD1
:1027E0007411F0C2071208039000FBE06006E4F0E9
:1027F0009001E0F0900166E07004A3E064017015C0
:10280000900166F0A3F09001AB7407F0A374D0F0D0
:10281000E49001E0F030040CC2049001E37401F094
:10282000A374F4F022787FE4F6D8FD758126023097
:102830004F020000023121E493A3F8E493A3400384
:10284000F68001F208DFF48029E493A3F85407240A
:102850000CC8C333C4540F4420C8834004F45680CA
:102860000146F6DFE4800B0102040810204080904E
:1028700037C5E47E019360BCA3FF543F30E50954A3
:102880001FFEE493A360010ECF54C025E060A84072
:10289000B8E493A3FAE493A3F8E493A3C8C582C869
:1028A000CAC583CAF0A3C8C582C8CAC583CADFE93E
:1028B000DEE780BEE49001BDF0A3F0200A03023100
:1028C0002020007CC20A9001F4E0902E12E0FFA3C9
:1028D000E09001BDCFF0A3EFF09001BDE0FFA3E0D9
:1028E0009001BBCFF0A3EFF0E4FF12371C12353A92
:1028F0009001BDCDF0A3EDF0EF64014E9001BD70ED
:102900000812352112355F8006123521123569E033
:102910003E9001B9F0A3EFF09001B9E0FEA3E0FF13
:102920001235499001F4E09001BBE0FFA3E0902E46
:1029300012CFF0A3EFF09001E37403F0A37420F042
:102940002253A87F1238CC1225AD1236DC1208169D
:1029500043A880E4F58D9000F17420F0122F72905E
:1029600001E0E014601514601714603814604A2404
:102970000470E0122E3C12080380D8122CDB803148
:10298000123852900020E0FF64206008EF6421605C
:1029900003123229900025E0641070B79001E074B2
:1029A00004F080AF1211189001E37403F0A37420B7
:1029B000F09001E07402F0809A12360D900025E04C
:1029C0006410608F120803808A9001C2EFF0E4A3C4
:1029D000F09001C2E0FFA3E0C39F502E121AD21262
:1029E00038FA900162EEF0A3EFF08E12F513C8747E
:1029F0000AC87400FCE4FDFB7A00790CFE7F081223
:102A00000D7F9001C3E004F080C71228EF90010011
:102A1000EEF0A3EFF0900160122CD4900133E09F10
:102A2000FF900132E09EFE1239287C007D05120DD8
:102A3000B7900130ECF0A3EDF0900160E0FFA3E06F
:102A4000900132CFF0A3EFF022308A779001E1E0DD
:102A50007002A3E0706D900166E07002A3E0706305
:102A6000F5B2758D20438D20758D8043A808D2AFB7
:102A7000F58B90012CE0FEA3E0FF4E6005758E50B3
:102A80008003758EFE20042F20092CE5DB54047092
:102A900026758AA4200920E5DB5404701AF5867592
:102AA0008703000000758601EF4E60047F288002D6
:102AB0007F7F7E00121D66758B01758A3053A8F7E3
:102AC0001238B0229001F5E014601B14603D24021E
:102AD000705430030D9001F57401F0D202D200124F
:102AE00038F0C20180409001F1E07002A3E0700272
:102AF000C2022003319001F57402F0D201C202C279
:102B0000009001F1F0A37458F0801B9001F1E07087
:102B100002A3E070119001F5200303F08006740118
:102B2000F01238F0C20120010330020A900025E0C3
:102B300064106002D20722E4FEEEC394077480940E
:102B40008050339001F4E0FDEE75F003A42428F5E5
:102B500082E4342EF583E5822DF582E43583123547
:102B60007EFDEE75F003A42427F582E4342E1235A1
:102B7000A7EDF00E80C3EF702D9001F4E0FF7E0012
:102B8000700A900147E07002A3E06010EF64014E0C
:102B90007014900149E07002A3E0700A9001F4E023
:102BA000902E217412F0227E007F137D007B017A2B
:102BB0000179F7121097E4FBEBC3940174809480C1
:102BC00050519001F4E0FFEB75F00AA42434F58233
:102BD000E43439F583E5822FF582E43583F583E427
:102BE00093FFE4FCFDFE122A6612100F122A6612F1
:102BF0000FF7EF04F87E007401088005C333CE336D
:102C0000CED8F9FFEE3395E0FDFC122A9912100F91
:102C10000B80A5229001E5E07004A3E0640170112F
:102C2000900007E06004D28AE4F0E49001E5F0A3AC
:102C3000F0900036E0FF9000FFE06F603D900036BE
:102C4000E0FD9000FFF0900007E09001F6F0540FD7
:102C5000F0ED7E0064207005E04420800CEF6410ED
:102C60004E700B9001F6E04410F0900007F0C28A1D
:102C70009001E57403F0A374E8F022CFF0EFA3F025
:102C8000900105121058020E03C3FF90017EE09FD1
:102C900090017DE095F02290011DE0FEA3E0FF226F
:102CA00090011DE0FFA3E0CF900195F0A3EFF0228B
:102CB0009001BCE0941E9001BBE094002290019D25
:102CC0007413F0A37488F0A3E4F0A322E4F0A3F05B
:102CD000A3F0A3F022FF90017DE5F0F0A3EFF02236
:102CE0009001B97408F0A3E4F0A3743FF0A374DF7B
:102CF000F0E4FDFCF9758A10538AEF009001B9E009
:102D0000FEA3E02DF582EE3CF583E493FF69F90D17
:102D1000BD00010CBC37E5BDDFE29001BBE0FEA3C6
:102D2000E0F5828E83E493FFE96F700890000174F0
:102D30000DF08005E4900001F0758A30538AEF00B1
:102D400022E0FEA3E0FF7C007D0A020DA59001C0F9
:102D5000E0902E1075F00202104C9001F4E0FF7E1E
:102D600000902E12E0FDA3E022900139121058EEDF
:102D70008FF0020E6675F002EF902E1002104C904C
:102D8000014AE02FFF90014922900148E02FFF9077
:102D90000147229001F4E02411F582E43408F58320
:102DA000E5822FF582E43583F583E493229001F4E4
:102DB000E02425F582E43402F583E022121003902A
:102DC000015CE0FEA3E022F583E4932420F582E495
:102DD000342EF583229001C7020FF7120E85900161
:102DE000C702100FE49001B9F0A3F0758A10538A5E
:102DF000EF00122DE475EA81E4F5F6F5F475F308B9
:102E0000F5F275EB0700E5EC30E7FBAFF3EFFEAD55
:102E1000F2EDFF900136121058EE8FF0120E66E4BC
:102E2000F5EC75EB30758A30538AEF00229000255F
:102E3000E06410703FF5B2758D20438D20538D7F77
:102E400053A8F7F58BE5DB54047013200910F58ABD
:102E5000F586758703000000758601758A30758BCD
:102E6000019001F37401F09001E37403F0A3742066
:102E7000F01238B022C2D5E830E70FB2D5E4C39BD8
:102E8000FBE49AFAE499F9E498F8EC30E717B2D544
:102E900012368B120F2BE4C39BFBE49AFAE499F9E8
:102EA000E498F88003120F2B30D50DE4C39FFFE4A4
:102EB0009EFEE49DFDE49CFC22E4FFEFC3940D74B0
:102EC000809480502E9001F4E0FEEF75F003A4246E
:102ED00001F582E4342EF583E5822E123583FEEF70
:102EE00075F003A42400F582E4342E1235A7EEF029
:102EF0000F80C8902F56E0902E2BF022E4F5DA7563
:102F0000DA4043DA2030881375D74075D6409001F7
:102F1000F404F090001574C9F0801175D74275D68D
:102F200042E49001F4F090001574CAF05392FE75DB
:102F3000DA5843A80275B80275F802229001BFEF73
:102F4000F01238939001BFE0FF1233179001BFE0F9
:102F5000FF9001F4E02411F582E43408F583E58262
:102F60002FF582E43583F583E493FF1226DC90018C
:102F7000BFE0FF02390B9001BBEFF07E007F10EE47
:102F8000C0E0EFC0E07D00E075F010A4240AF97401
:102F90000235F0FA7B01D0E0FFD0E0FE12109790EE
:102FA00001BBE0122BED740BF0A374B8F02290017A
:102FB00057E02448FF900156E034F4FEC3900161CD
:102FC000E09F900160E09E5014900166E07002A3C3
:102FD000E0701190016604F0A374F4F022E4900113
:102FE00066F0A3F022C1094202250206C10A41018E
:102FF000F6004101F5004101F400C103C101C10027
:10300000C102C105011600C104C106C108C10741C2
:1030100000FF10430220010223009001C17401F05F
:103020009001C1E0C3122C6750167F011231A91222
:1030300021EC900102122C2B9001C1E004F080E001
:10304000E49001E9F0A3F02290011DE0FEA3E0FF6F
:103050007C0012106AE47B64FAF9F8120F2B9001DD
:1030600091EEF0A3EFF0A3E022900220121058029C
:103070000E0312082E7F011231A91221EC900102D9
:10308000122C2B1215091227FD1223311233F412C0
:10309000378E0230947E007F027D007B017A0179B9
:1030A000581210977E007F027D007B017A01795CC7
:1030B000021097EFF87401088002C333D8FC42ABCA
:1030C00012357390080E93F4529152935391DF226C
:1030D000E5B254016006E5A85410700F75B2927500
:1030E000B67CE4F5B743B20143A81022758A305389
:1030F0008AEF758601758F05E4F5AB75AC0F759198
:103100003E759201D28A227E007D007B01021097DB
:103110009001F104F0A37458F022900160E0FEA346
:10312000E0FF90015EEEF0A3EFF0221235739008FD
:103130000E9342914288439120227816E6FF2400A4
:10314000F582E43400F58322EE30E707C3E49FFF05
:10315000E49EFE2203030019001E001400190096CD
:1031600000960701F40000000000000000000000CD
:10317000000000000000000000000000000000004F
:10318000000000000000000000000000000000003F
:10319000000000000000000000000000000000002F
:1031A000000000000000000000000000000000001F
:1037F0000000000000000000000000000000008A3F
:1038000000000000000000000000000000000000B8
:1038100000000000000000000000000000000000A8
:00000001FF
